:103B52000FAA0FA50F9F0F9A0F940F8D0F870F803B
:103B62000F780F710F680F600F570F4E0F450F3B05
:103B72000F300F250F1A0F0E0F020EF50EE80EDB97
:103B82000ECC0EBE0EAE0E9F0E8E0E7D0E6C0E5A1B
:103B92000E470E340E200E0C0DF70DE20DCB0DB5B7
:103BA2000D9D0D850D6D0D540D3A0D200D050CE981
:103BB2000CCE0CB10C940C760C580C3A0C1B0BFB73
:103BC2000BDB0BBB0B9A0B790B570B350B130AF163
:103BD2000ACE0AAB0A870A640A400A1C09F809D409
:103BE20009B0098C09670943091F08FB08D608B206
:103BF200088E086A0846082307FF07DC07B90796FC
:103C020007730751072F070D06EC06CA06AA068995
:103C120006690649062A060A05EC05CD05B0059295
:103C220005750558053C0520050504EA04CF04B5D1
:103C3200049C04820469045104390422040B03F431
:103C420003DE03C803B2039D038903750361034DB9
:103C5200033B03280316030402F202E102D102C06D
:103C620002B002A002910282027302650257024967
:103C7200023C022F02220216020901FD01F201E6B4
:103C820001DB01D001C601BB01B101A7019D019475
:103C9200018B0182017901700168016001580150B4
:103CA2000148014101390132012B0125011E011890
:103CB2000111010B010500FF00FA0ECF0EBB0EA78A
:103CC2000E920E7C0E650E4D0E340E190DFE0DE198
:103CD2000DC40DA50D850D640D420D1E0CFA0CD4FC
:103CE2000CAE0C860C5D0C330C080BDC0BB00B829B
:103CF2000B540B250AF50AC40A930A610A2F09FD1F
:103D020009CA09960963092F08FC08C808950861C1
:103D1200082E07FB07C8079607640733070206D277
:103D220006A206730645061705EA05BF059305694F
:103D32000540051704F004C904A3047E045A04379D
:103D4200041503F403D303B403960378035B033F20
:103D52000324030A02F002D702BF02A80292027CE5
:103D620002670253023F022C021A020801F701E61F
:103D720001D601C701B801A9019C018E018101741C
:103D82000168015D01510146013C01320128011F18
:103D92000115010D010400FC00F400EC00E500DE59
:103DA20000D700D000CA00C300BD00B800B200AD09
:103DB20000A700A2009E009900940090008C00874A
:103DC20000840080007C007800750072006E006B39
:103DD2000068006500620060005D005A00580055EE
:103DE20000530051004E004C004A00480046004477
:103DF20000430041003F003E003C003A00390037DA
:103E020000360035003300320031002F002E002D25
:103E1200002C002B002A002900280027002600255C
:103E22000024002300010C01010602011E030A9670
:103E320004013205050506006407010108000009B6
:103E4200015A0A01040B00030E01010F00011200C6
:103E52006413010114013C1501FA1664FA17FFFFFD
:103E62001D00072000072400022632962701012C9C
:103E7200000130030332010333000235FFFF360332
:103E8200073CFFFF3DFFFF180002191E461A000201
:0F3E92001B00022D32C82E00012F013CFAFAFA54
:10004800E50C902208F8282873803475E700A21080
:10005800B34008E5B54408F5B58006E5B554F7F5AD
:10006800B575E710801975E700A210B34008E5B52B
:0F0078004402F5B58006E5B554FDF5B575E71002
:0922080002005102005302006EB5
:100087002290083DE0900043F090083EE090004A3F
:10009700F090083FE090004BF0900840E090004E51
:1000A700F0900841E090004FF0900842E090005235
:1000B700F0900843E0900053F0900844E090005E11
:1000C700F0900845E0900060F0900846E0900064EA
:1000D700F0900847E0900066F0900848E0900067CD
:1000E700F0900849E0900068F090084AE0900069B5
:1000F700F090084BE090006CF090084CE090006D99
:10010700F090084DE090006FF090084EE09000707E
:10011700F090084FE090007CF0900850E090007D50
:10012700F0900851E090007EF0900852E090007F38
:10013700F0900853E0900080F0900854E090008120
:10014700F0900855E0900082F0900856E090008308
:10015700F0900857E0900085F0900858E0900086EE
:10016700F0900859E0900087F090085AE0900088D6
:10017700F090007CE090002CF090007DE090002D46
:10018700F090007EE090002EF090007FE090002F2E
:10019700F0900080E0900030F0900081E090003116
:1001A700F0900082E0900032F0900083E0900033FE
:1001B700F0900085E0900028F0900086E0900029FC
:1001C700F0900087E090002AF0900088E090002BE4
:1001D700F07441900111F07442900112F07436905E
:1001E7000113F07430900114F07420900115F0742D
:1001F70041900116F07437900117F074369001188A
:10020700F07431900119F0744590011AF074209040
:10021700011BF0743690011CF0745390011DF074AB
:100227007090011EF0746490011FF0900440E090FC
:100237000480F02290083AE0FEA3E0FF7463BE005A
:1002470010D39F400C903E2612001EE493F5998030
:100257001290083AE0FEA3E0FF903E2612001EE44B
:1002670093F59990083A12000E90083AE0FEA3E041
:10027700FF747B6F4E70037567002290005EE0B4D9
:100287000208740190005EF0D20A757002A206B3EC
:100297004016900126E0700C900127E0700690014F
:1002A70028E060028002C206900126E0B4300F9079
:1002B7000127E0B44708900128E0643B600280040E
:1002C700D2078002C207E549B40102800302039FF7
:1002D70090007CE090002CF090007DE090002DF0E5
:1002E70090007EE090002EF090007FE090002FF0CD
:1002F700900080E0900030F0900081E0900031F0B5
:10030700900082E0900032F0900083E0900033F09C
:10031700900085E0900028F0900086E0900029F09A
:10032700900087E090002AF0900088E090002BF082
:10033700900065E0B40117900000740FF0A374FFFC
:10034700F0900002E4F0A3F07402900065F09000D2
:1003570065E0B40341900002E0FEA3E0FF900000D7
:10036700E0FCA3E0FD120003741012407174081240
:100377004063EF900064F0EF700674FF900064F044
:100387007400900065F0900001E090004AF0900042
:1003970000E090004BF0800990006DE07003754914
:1003A700017E897F89900043E08E048F05FF12400C
:1003B700538C338D3490004FE075F0FAA4FFAEF004
:1003C70090004EE08E048F05FF1240538C378D3816
:1003D70090003BE0F54F900038E0FE900055E0B507
:1003E7000618900037E0FE900054E0B5060C900028
:1003F70036E0FE900045E06E606F900055E07006B5
:10040700900054E060067400900045F0900055E0BD
:10041700B402089000347401F08005900034E4F0D1
:10042700900054E0B402089000357401F080059004
:100437000035E4F0900054E06006900035E060027B
:100447008005754F058003754F06E54AB54902D209
:100457000A900054E0900037F0900055E090003883
:10046700F0900045E0900036F0740090008AF07438
:100477000190008BF0740190008CF0740090008D57
:10048700F0740190008EF0740090008FF07401906A
:100497000090F07400900091F07401900092F07455
:1004A70001900093F07400900094F074019000950F
:1004B700F07400900096F07401900097F07400902B
:1004C7000098F07401900099F0740190009AF0740C
:1004D7000090009BF0740190009CF0740090009DC8
:1004E700F0740190009EF0740090034EF074019038
:1004F700034FF07401900350F07400900351F074AF
:1005070001900352F07400900353F0740190035468
:10051700F0740190038EF0740190038FF0740190D2
:100527000390F07400900391F07401900392F074BB
:1005370000900393F07401900394F074019003CE3C
:10054700F074009003CFF074019003D0F074009022
:1005570003D1F074019003D2F074009003D3F074C8
:10056700019003D4F0740190040EF0740090040F0E
:10057700F07400900410F07400900411F07401906E
:100587000412F07400900413F07401900414F074D2
:100597000190044EF0740090044FF07400900450E2
:1005A700F07401900451F07400900452F0740190BB
:1005B7000453F07400900454F0740190048EF074A6
:1005C7000190048FF07400900490F07401900491EE
:1005D700F07400900492F07401900493F07400900A
:1005E7000494F012223222C293C294C292C287C2EA
:1005F70090755200755300C203E5B554FBF5B57508
:100607004406E54404F54590003BE0F54F9000268D
:10061700E4F0C205900039E4F0E5B554FEF5B59075
:100627000026E4F0755100C28E758D00758B00753C
:100637004100752600752500D28EC296C295C2A0CC
:10064700C297C2A2E5B554DFF5B5E5B554BFF5B518
:10065700E5B554EFF5B5E5B5547FF5B5E5B554F710
:10066700F5B5E5B554FDF5B522755900755800AED9
:1006770058AF597462BE00039F500302072D903E86
:100687002612001EE49390003A1240890FBF000122
:100697000EE0FC903E2612001EECFEE493FFEEC334
:1006A7009F5026AE58AF590FBF00010E903E26123D
:1006B700001EAE58AF59E493FC903E2612001EE48C
:1006C7009390003A124089ECF0AE58AF59903E260D
:1006D70012001EE49390003A124089E0FC903E28F5
:1006E70012001EECFCE493FDECD39D4019903E28CC
:1006F70012001EE493FC903E2612001EE493900025
:100707003A124089ECF0AE58AF5974022FFF5001EE
:100717000E8E588F597859740126F6500418E4360E
:10072700F6400302067622755900755800AE58AF99
:10073700597417BE00039F50030207FB903E8912AE
:10074700001EE49390003A1240890FBF00010EE0AB
:10075700FC903E8912001EECFEE493FFEEC39F500F
:1007670026AE58AF590FBF00010E903E8912001EEA
:10077700AE58AF59E493FC903E8912001EE4939063
:10078700003A124089ECF0AE58AF59903E891200FA
:100797001EE49390003A124089E0FC903E8B1200D1
:1007A7001EECFCE493FDECD39D4019903E8B1200A8
:1007B7001EE493FC903E8912001EE49390003A12C7
:1007C7004089ECF0AE58AF5974126F4E70067559E8
:1007D70018755800AE58AF5974022FFF50010E8E8E
:1007E700588F597859740126F6500418E436F640A4
:1007F700030207342212067012072E220542220531
:1008070041220543C2CF2290F800E49364066002B8
:1008170080FE75840175A70075FF8090083CE4F0A1
:1008270075C91075A70F75A1C775A70075D900758C
:10083700CEFF75A70F75F1FE75F2FF75F33775F4E7
:100847007875A4BA75A5FF75A60775AE0075AFFFD5
:1008570075D48175D5FF75D6FF75D7FFC296C2953A
:10086700C2A0C297C2A2E5B554EFF5B5E5B5547F6E
:10087700F5B5E5B554F7F5B5E5B554FDF5B575A787
:100887000075A20175A14775F80975BC0175BE040D
:1008970075BD6C75BE0775BDA075BE0875BD0175C4
:1008A700BC0075BB1875BC2075BA0875E88075D192
:1008B7001375A70F75E10575E20075C740759700B9
:1008C700759780740A1240437597C0E59754207056
:1008D7000280F8758F0275A700D2AF75980075A9C9
:1008E7000C75A70F75AB4375ADFB75AC1E75A700EF
:1008F700758911758E00758C00758A00D2A9D28C06
:10090700758D00758B00D2ABD28E75CD0075CC007E
:1009170075CA0075CB00D2ADC2CFD2CA7591047526
:1009270092007593CD75EF0675D94075CF01900884
:100937003AE4F0A3F0756700756800C299C20C121B
:1009470005EE7509C875080012236875A70FE5FC41
:10095700900015F0E5FB900016F0E5FA900017F00F
:10096700E5F9900018F075A70090F800E493F557A3
:100977001224871229C190F807E493900022F0907F
:100987000022E04408900022F0900022E054FE90FC
:100997000022F012008890085BE0900126F0900892
:1009A7005CE0900127F090085DE0900128F090014D
:1009B70026E0700C900127E07006900128E06002A5
:1009C7008004C2068002D206754901754A01740384
:1009D700900037F01207FC7400900065F0740090E7
:1009E700006EF01202827406900008F07400900006
:1009F70009F0740290000AF090F802E49390000B5B
:100A0700F090F803E49390000CF090F804E49390CE
:100A1700000DF0740590000EF0740490000FF07450
:100A270003900010F07406900011F0740290001209
:100A3700F090F805E493900013F090F806E4939093
:100A47000014F0740090001CF0740090001DF07406
:100A57000090001EF0740090001FF07400900020BA
:100A6700F07400900021F074FF900023F0A2B6B359
:100A77009200A2B3B39201756D00743A90073AF0F1
:100A870074FD90073BF0C20A900024E4F0754B0018
:100A9700752400752300753E00752A0075290075B9
:100AA7003F0075460075470075450175550075543B
:100AB700007556CD754800900027E4F0753B00752A
:100AC7003C00753D00753A00753900754E00900081
:100AD7000474FDF0A374E8F0900024E4F0746490CB
:100AE7000025F0754200E5B554DFF5B5C2A1C20B8C
:100AF700C29112233BC203D2B0D2B7D2A7D2A6D299
:100B0700B1D2A37E017F0090004BE01240719000AC
:100B17004AE02FFF50010E900000EEF0A3EFF0EF38
:100B2700D394FFEE940F4007900000E4F0A3F090F9
:100B37000064E0700674FF900064F0D29CD2EC75FC
:100B4700CF01A298B34005C298122D6DE5676006E4
:100B5700A299B3B340028005C299123183E5686454
:100B6700016005E568B4040280D5E542D3940540E9
:100B77000CE54BC394C85002054B754200E556C3BC
:100B870094F0501A785412003FAE54AF55EFD394F7
:100B9700E8EE940340080556755500755400C28E5B
:100BA7007E047F00E541124071E58D75F004A4FDD8
:100BB700ACF0EF2DFDEE3CFCE58B75F04084FF7E3D
:100BC70000ED2FFFEC3EFE8E258F26D28EA2B6308B
:100BD7000001B35003020D53A2B6300001B3500316
:100BE700020D53A2B640730546A20C400575FFA03F
:100BF700D20CE5B54401F5B5900025E4F09000432B
:100C0700E0C395465052E5264525600F7C897D89CE
:100C1700AE25AF26123EA18E238F24AE23AF24E547
:100C27003E2FFF50010E74011240638E238F2485DF
:100C3700243E754601C28E758D00758B0075410087
:100C4700D28E7403BE00039F50069000267401F0F5
:100C5700E56DB40D03756D00D200A2B6B350030263
:100C67000D53900025E4F0C200900057E060077430
:100C770001F5081232C490005AE060097402F508C1
:100C87001232C48013A20BB34008E5B54402F5B590
:100C97008006E5B554FDF5B5E548B40708E5B54464
:100CA70080F5B58006E5B5547FF5B5A203B34008D6
:100CB700E5B54440F5B58006E5B554BFF5B59000F8
:100CC70045E06004D20B8002C20B900035E0B4010E
:100CD70008E5B54420F5B58006E5B554DFF5B590D0
:100CE7000034E0B40104D2A18002C2A1A205B3403E
:100CF70004D2918002C29190000EE0FE90000BE0BA
:100D0700C39E400990000BE0D39408400974FB9000
:100D17000024F01205EE90000CE0601590000CE046
:100D2700FE90000AE06E600974FC900024F0120542
:100D3700EE90000DE0601590000DE0FE90000FE0D2
:100D47006E600974FE900024F01205EEC2CA7E019F
:100D57007F00E543124071E5CD2FFF50010E8E272E
:100D67008F28D2CA900068E0B40148900004E0FCE4
:100D7700A3E0FDEFC39DEE9C4039B204E52A452967
:100D87006013A204B34008E5B54404F5B58006E551
:100D9700B554FBF5B5900004E0FEA3E0FF90000614
:100DA700E0FCA3E0FDEF2DFDEE3CFC900004ECF031
:100DB700A3EDF0A2B3300101B35003020EF3A2B3C7
:100DC700300101B35003020EF3A2B35003020EEC3D
:100DD7000547A20C400575FFA0D20CE5B54401F507
:100DE700B5900025E4F090004EE0C395474003021C
:100DF7000EEAE5284527600F7CEA7D60AE27AF281D
:100E0700123EA18E298F2AAE29AF2A90004FE012F9
:100E1700407174FF8E048F05FF1240538C298D2A71
:100E2700E53F2DFD50010C74018C068D07124063C0
:100E37008E298F2A852A3FA205B340157464124074
:100E470071900053E08E048F05FF1240538C298D5B
:100E57002A754701900004E0FEA3E0FFAC27AD2808
:100E6700120003900004EEF0A3EFF07AFF7BFF90EF
:100E77000067E08A048B05FF124053AE27AF28EDC9
:100E8700D39FEC9E4023900067E012407174828EDE
:100E9700048F05FF124053900069E0FF1240539002
:100EA7000006ECF0A3EDF0802DAE27AF2874828EFC
:100EB700048F05FF124053900067E08C068D0712E0
:100EC7004071900069E08E048F05FF124053900037
:100ED70006ECF0A3EDF0C2CA75CD0075CC007543E2
:100EE70000D2CAD201A2B3B34002C201900026E0E9
:100EF700B40107E548C39406400302151FE5519066
:100F07002211F8282873900045E0C3940240030299
:100F17001061E544D394015003021061E54475F074
:100F270040A4FFAEF09002FE12001EE0C3953C50B5
:100F370018E54475F040A4FFAEF09002FD12001EC4
:100F4700E0F52E752D00021061E54475F040A4FF11
:100F5700AEF09002FC12001EE0C3953C4003020F66
:100F6700FDE54475F040A4FFAEF09002FD12001EAF
:100F7700E54475F040A4FFAEF0E0FC9002FB1200E0
:100F87001EECFEE0FFEEC39FFEE5448E0475F040C5
:100F9700A4FFAEF09002FC12001EE0F404253C8C86
:100FA7000088F0A4FFAEF0E5448F048E0575F0408D
:100FB700A4FFAEF09002FE12001EE54475F040A4B7
:100FC700FFAEF0E0FA9002FC12001EEAFEE0FFEE30
:100FD700C39FFECDCCCD8E07124053E54475F0403C
:100FE700A4FFAEF09002FB12001EE02DFD50010C95
:100FF7008C2D8D2E8064E54475F040A4FFAEF090F3
:1010070002FB12001EE54475F040A4FFAEF0E0FCC1
:101017009002FA12001EECFEE0FFEEC39F853CF043
:10102700A4FFAEF0E5448F048E0575F040A4FFAE33
:10103700F09002FC12001EE0FECDCCCD8E071240D0
:1010470053E54475F040A4FFAEF09002FA12001E7B
:10105700E02DFD50010C8C2D8D2E75510102151FB1
:10106700900045E0C39402400302121590003BE054
:10107700D3954450030211BDE54475F040A4FFAE7B
:10108700F090030412001EE0C3953C5018E5447528
:10109700F040A4FFAEF090030312001EE0F52C759C
:1010A7002B000211BDE54475F040A4FFAEF090039C
:1010B7000212001EE0C3953C4003021159E5447536
:1010C700F040A4FFAEF090030312001EE54475F054
:1010D70040A4FFAEF0E0FC90030112001EECFEE01E
:1010E700FFEEC39FFEE5448E0475F040A4FFAEF00B
:1010F70090030212001EE0F404253C8C0088F0A443
:10110700FFAEF0E5448F048E0575F040A4FFAEF006
:1011170090030412001EE54475F040A4FFAEF0E012
:10112700FA90030212001EEAFEE0FFEEC39FFECD17
:10113700CCCD8E07124053E54475F040A4FFAEF0C6
:1011470090030112001EE02DFD50010C8C2B8D2CFD
:101157008064E54475F040A4FFAEF09003011200EF
:101167001EE54475F040A4FFAEF0E0FC90030012CA
:10117700001EECFEE0FFEEC39F853CF0A4FFAEF03F
:10118700E5448F048E0575F040A4FFAEF09003028E
:1011970012001EE0FECDCCCD8E07124053E54475FC
:1011A700F040A4FFAEF090030012001EE02DFD50AA
:1011B700010C8C2B8D2CE544B40123E54FD394010E
:1011C700401CE54804D395444014E53CC3940550BE
:1011D7000D90034BE0A829B80006952A400280032A
:1011E700754402E544B54F2290003BE0D395444057
:1011F70019E54475F040A4FFAEF090030312001EFA
:10120700E0A823B80006952440028002054F7551D7
:101217000202151F900045E0B4022AE54475F0402C
:10122700A4FFAEF090030312001EE0F52C752B000F
:10123700E54475F040A4FFAEF09002FA12001EE0FC
:10124700F52E752D00900045E0B4030F90003DE0AA
:10125700F52C752B00752E00752D007551030215A1
:101267001FE54475F040A4FFAEF090030C12001E7A
:10127700E0C3954B400302133D900034E07036E520
:1012870044D394014029AE23AF24AC2DAD2EEDD32A
:101297009FEC9E401AE54475F040A4FFAEF0900322
:1012A7000A12001EE0A829B80005D3952A5002802B
:1012B7000215448034E544D394024029AE23AF2479
:1012C700AC2DAD2EEDD39FEC9E401AE54475F04052
:1012D700A4FFAEF090030A12001EE0A829B800058B
:1012E700D3952A500280021544E544B54537E544B5
:1012F700C3954F5030E54804D395444028AE23AFFB
:1013070024AC2BAD2CEFD39DEE9C4019E54475F032
:1013170040A4FFAEF090030B12001EE0A829B8000E
:1013270006952A400280020544C290E5446545605F
:1013370005C203754B0075510402151FE54475F08E
:1013470040A4FFAEF090030612001EE0B40117E5BB
:101357004475F040A4FFAEF090030C12001EE02489
:101367000AC3954B4003021413753064752F00A20E
:1013770003B3500B90004CE02405C3953C40030297
:101387001413E54475F040A4FFAEF0900309120072
:101397001EE0C3953C4064E54475F040A4FFAEF001
:1013A70090030812001EE54475F040A4FFAEF0E07C
:1013B700FC90030712001EECFEE0FFEEC39F853C86
:1013C700F0A4FFAEF0E5448F048E0575F040A4FF4E
:1013D700AEF090030912001EE0FECDCCCD8E0712B1
:1013E7004053E54475F040A4FFAEF09003071200A8
:1013F7001EE02DFD50010C8C2F8D30AE23AF24AC99
:101407002FAD30EFD39DEE9C4002D20375510502FC
:10141700151FE544B40109900045E0C39402400359
:101427000214E7900344E0D3953C50030214E7907D
:101437000342E0C3953C5040900343E0FE900341D4
:10144700E0F4042EFE900342E0F404253C8E00886D
:10145700F0A4FFAEF0900344E0FC900342E0F404F4
:101467002C8E048F05FF124053900341E02DFD5051
:10147700010C8C2B8D2C802C900341E0FE900340B7
:10148700E0F4042E853CF0A4FFAEF0900342E08E1A
:10149700048F05FF124053900340E02DFD50010CCF
:1014A7008C2B8D2CE544C3954F5030E54804D395DC
:1014B700444028AE23AF24AC2BAD2CEFD39DEE9C3C
:1014C7004019E54475F040A4FFAEF090030B1200FD
:1014D7001EE0A829B80006952A4002800375440239
:1014E700900034E0B40106E54464016002800375AE
:1014F7004402E54465456005C203754B0090003919
:10150700E0B40107E54BD3940A50028008900039F4
:08151700E4F075440175510078
:10221100020F0D02106702121B0212680213430221
:0222210014198E
:10151F0090003CE02402A823B80007D39524400292
:10152F00C203900027E065486030E548B4070375B3
:10153F004B00E548B4050F900027E0D39405400613
:10154F00E54464016002800C754406900039740113
:10155F00F0754B00E548900027F0900026E0B401AD
:10156F0009900045E0C3940340030216EB9000344A
:10157F00E06003021634E544D39401403A900039F9
:10158F00E07034E54475F040A4FFAEF09003001214
:10159F00001EE0A823B8001FD39524401AE5447518
:1015AF00F040A4FFAEF090030B12001EE0A829B884
:1015BF000005D3952A500280021544E544D39401C7
:1015CF00402FE54475F040A4FFAEF09002FE1200EC
:1015DF001EE0C3953C501AE54475F040A4FFAEF0F1
:1015EF0090030A12001EE0A829B80005D3952A50CF
:1015FF000280021544E544D394014022E54804C318
:10160F009544501AE54475F040A4FFAEF090030ADC
:10161F0012001EE0A829B80005D3952A50028002B7
:10162F0015440216E0E544D39402403A900039E0A5
:10163F007034E54475F040A4FFAEF0900300120043
:10164F001EE0A823B8001FD39524401AE54475F077
:10165F0040A4FFAEF090030B12001EE0A829B800C3
:10166F0005D3952A500280021544E544D3940240D5
:10167F002FE54475F040A4FFAEF09002FE12001E5D
:10168F00E0C3953C501AE54475F040A4FFAEF090CE
:10169F00030A12001EE0A829B80005D3952A5002AC
:1016AF0080021544E544D394024022E54804C395D3
:1016BF0044501AE54475F040A4FFAEF090030A12AF
:1016CF00001EE0A829B80005D3952A500280021504
:1016DF0044E54465456005C203754B0090004CE03E
:1016EF00D3953C5009900040E0C3953C5002C20393
:1016FF00900045E07003021952A2A5B34008A2A4BE
:10170F00B3400302193BAE31AF327441D39F749C87
:10171F009E4005783112003FAE31AF32EFB48806EC
:10172F00EEB413028003021916A2A550030217D9B3
:10173F00900045E0B4010B90003BE0D3954F400281
:10174F00054F900045E0B40254E54475F040A4FF06
:10175F00AEF090030C12001EE0C3954B503F90006B
:10176F003BE0D395444021E54804D395444019E527
:10177F004475F040A4FFAEF090030012001EE0A8E5
:10178F0023B80006952440028002054490003BE0F8
:10179F00F54FE54465456005C203754B0090004564
:1017AF00E0B4032690003BE0D395444008E548049D
:1017BF00D3954450028002054490003BE0F54FE57D
:1017CF004465456005C203754B00A2A4500302197E
:1017DF0016900045E0B4016E900034E07035E5449A
:1017EF00D394014029E54475F040A4FFAEF0900377
:1017FF000A12001EE0A829B8000FD3952A400A1537
:10180F0044754B0085444F800385444F8003754FCB
:10181F00018033E544D394024029E54475F040A498
:10182F00FFAEF090030A12001EE0A829B8000FD3F4
:10183F00952A400A1544754B0085444F8003854413
:10184F004F8003754F02900045E0D394015003027F
:10185F00190AE54475F040A4FFAEF090030C120096
:10186F001EE0C3954B400302190A900034E070410B
:10187F00E544D394014034E54475F040A4FFAEF045
:10188F009002FD12001EE0A823B8001FD39524403C
:10189F001AE54475F040A4FFAEF090030A12001E43
:1018AF00E0A829B80005D3952A500280021544807C
:1018BF003FE544D394024034E54475F040A4FFAEB5
:1018CF00F09002FD12001EE0A823B8001FD395244C
:1018DF00401AE54475F040A4FFAEF090030A1200E1
:1018EF001EE0A829B80005D3952A5002800215449E
:1018FF00E54465456005C203754B00E548B4070430
:10190F00054E8003754E0090006DE0B4010EAE31B0
:10191F00AF32EF64407005EE649C6002800EA2A5AA
:10192F004003754901A2A44003754902A2A5B3B3B0
:10193F005006A2A4B3B34002800675320075310081
:10194F00021A48A2A5B34008A2A4B34003021A3456
:10195F00AE31AF327441D39F749C9E4005783112E3
:10196F00003FAE31AF32EFB48806EEB413028003FE
:10197F00021A34A2A54077900054E06062900035BF
:10198F00E0B40107900035E4F08006900035740153
:10199F00F0900035E07005754F058003754F069088
:1019AF000035E0B40108E5B54420F5B58006E5B58E
:1019BF0054DFF5B5E544B4061AE54475F040A4FFCD
:1019CF00AEF090030A12001EE0A829B80005D395C7
:1019DF002A50028008754405C203754B00800375B9
:1019EF004F06E548B40704054E8003754E00A2A4C8
:1019FF004033900055E06021900034E0B40107902F
:101A0F000034E4F080069000347401F0900034E06C
:101A1F00B40104D2A18002C2A1E548B40704054E67
:101A2F008003754E00A2A5B3B35006A2A4B3B34072
:101A3F00028006753200753100E549654A600690EF
:101A4F00006EE06002802CE549902223F82828736D
:101A5F0080121229C1800D122AAC8008122B978098
:041A6F0003122C82B0
:0F222300021A5F021A61021A66021A6B021A701F
:101A730012008812028285494A741B900024F0E503
:101A830048C394065005E544B54503021B8DC203C4
:101A9300E54475F040A4FFAEF090030E12001EE083
:101AA30030E003D38001C39296E54475F040A4FF70
:101AB300AEF090030F12001EE030E003D38001C3A9
:101AC3009295E54475F040A4FFAEF0900310120028
:101AD3001EE030E003D38001C392A0E54475F040DB
:101AE300A4FFAEF090031112001EE030E003D38098
:101AF30001C39297E54FB40206E544640260028095
:101B030002D297E545B40506E54464046002800407
:101B1300C2A28019E54475F040A4FFAEF090031211
:101B230012001EE030E003D38001C392A2E54475A6
:101B3300F040A4FFAEF090031312001EE030E00368
:101B4300D38001C39208E54475F040A4FFAEF09042
:101B5300031412001EE030E003D38001C39209E5B1
:101B63004FC394045006E54F654460028002C209E6
:101B7300854445AE29AF2A7405BE00039F5007E58F
:101B83003CD3940550028002D290E544B40406E5A8
:101B93004B640A60028019E54475F040A4FFAEF07F
:101BA30090031212001EE030E003D38001C392A21F
:101BB30090005EE06058E53C75F00284FF7E009083
:101BC300013A12001EE0F54CE53D75F00A84FF7EF4
:101BD3000090023A12001EE0F54DE54C254DD394DA
:101BE30064400BE54C254DC39464F54C8003754C60
:101BF30000E54C75F00284FF7E008F4CEFC39433F5
:101C03005007EF24CDF54C8003754CFF801CE53C59
:101C130075F00284FF7E0090013A12001EE075F019
:101C23000284FF7E00EF24CDF54CE548D3940550A4
:101C330003021E4AC203E544D394015003021D1D4F
:101C4300E54475F040A4FFAEF090030A12001EE0D5
:101C5300A829B80007D3952A40021544E5446545F1
:101C63007003021D1AE54475F040A4FFAEF0900323
:101C73000E12001EE030E003D38001C39296E544C8
:101C830075F040A4FFAEF090030F12001EE030E0A9
:101C930003D38001C39295E54475F040A4FFAEF0F1
:101CA30090031012001EE030E003D38001C392A022
:101CB300E54475F040A4FFAEF090031112001EE05E
:101CC30030E003D38001C39297E54475F040A4FF4D
:101CD300AEF090031212001EE030E003D38001C384
:101CE30092A2E54475F040A4FFAEF09003131200F6
:101CF3001EE030E003D38001C39208E54475F04051
:101D0300A4FFAEF090031412001EE030E003D38072
:101D130001C39209854445021E4AE548B4065B9017
:101D23000098E030E003D38001C39296900099E0DD
:101D330030E003D38001C3929590009AE030E00332
:101D4300D38001C392A090009BE030E003D38001D5
:101D5300C3929790009CE030E003D38001C392A22A
:101D630090009DE030E003D38001C3920890009E71
:101D7300E030E003D38001C39209E548B4076890DB
:101D83000091E030E003D38001C39296900092E08B
:101D930030E003D38001C39295900093E030E003D9
:101DA300D38001C392A0900094E030E003D380017C
:101DB300C39297900095E030E003D38001C392A2D1
:101DC300900096E030E003D38001C392089000971F
:101DD300E030E003D38001C39209E54BD394144070
:101DE30003754CCD854445E548B4085B90008AE013
:101DF30030E003D38001C3929690008BE030E00380
:101E0300D38001C3929590008CE030E003D380012E
:101E1300C392A090008DE030E003D38001C392977A
:101E230090008EE030E003D38001C392A290008F34
:101E3300E030E003D38001C39208900090E030E0EB
:101E430003D38001C39209E595C3954C4004C29323
:101E53008002D293A203B34005E548B40703755645
:101E6300CDE595C395564004C2948002D294E53CD7
:101E730075F00284FF7E0090016C12001EE075F085
:101E83000284FF7E00EF24CDF552E595C3955250B1
:101E930006A208B3B340028004D2928002C292E544
:101EA3003C75F00284FF7E0090019E12001EE075D7
:101EB300F00284FF7E00EF24CDF553E595C39553DF
:101EC3005006A209B3B340028004D2878002C287BE
:101ED300E56DC3940D501DE56D75F00284AFF07E82
:101EE30000EF4E700512350A800AA2EDB34005C219
:101EF300ED12350AE54ED3940450030220C375CF87
:101F030001C293AE31AF327488D39F74139E4005E0
:101F1300A2A5B34014AE31AF327488D39F74139E1D
:101F23004005A2A4B340028048783112003FAE318D
:101F3300AF32EFB4883BEEB41337A2A5B350099088
:101F4300003BE0D395445002800405448011A2A5D0
:101F5300B3500890003BE0654460028002D203A2C4
:101F6300A4B35007E544D39401500280041544C23E
:101F730003A2A5B3B35006A2A4B3B340028006756F
:101F83003200753100E54465457003022045E544A0
:101F930075F040A4FFAEF090030E12001EE030E097
:101FA30003D38001C39296E54475F040A4FFAEF0DD
:101FB30090030F12001EE030E003D38001C392951B
:101FC300E54475F040A4FFAEF090031012001EE04C
:101FD30030E003D38001C392A0E54475F040A4FF31
:101FE300AEF090031112001EE030E003D38001C372
:101FF3009297E54475F040A4FFAEF09003121200EF
:102003001EE030E003D38001C392A2E54475F040A3
:10201300A4FFAEF090031312001EE030E003D38060
:1020230001C39208E54475F040A4FFAEF090031499
:1020330012001EE030E003D38001C39209C29485ED
:102043004445A20340057556CD80037556FFE595BB
:10205300C395564004C2948002D294E53C75F002C5
:1020630084FF7E0090016C12001EE075F00284FF75
:102073007E00EF24CDF552E595C395525006A20894
:10208300B3B340028004D2928002C292E53C75F061
:102093000284FF7E0090019E12001EE075F0028410
:1020A300FF7E00EF24CDF553E595C395535006A26B
:1020B30009B3B340028004D2878002C287021F01A2
:1020C300A20CB3500DAE25AF2674E8C39F74039ED4
:1020D3004002800575FFA0D20CAE25AF26EFD39446
:1020E30020EE944E50030221DC1205EEC28E758D54
:1020F30000758B00754100D28EC20375550075546F
:10210300007556CD75440675240075230075460089
:10211300754B00E5B554BFF5B5900045E06004D2BA
:102123000B8002C20B900035E0B40108E5B54420F2
:10213300F5B58006E5B554DFF5B5900034E0B4019C
:1021430004D2A18002C2A1A205B34004D2918002AD
:10215300C291900057E060077401F5081232C490F1
:10216300005AE060097402F5081232C48013A20B0E
:10217300B34008E5B54402F5B58006E5B554FDF571
:10218300B5E548B40708E5B54480F5B58006E5B57F
:10219300547FF5B590000474FDF0A374E8F0E56D89
:1021A300B40D03756D00752600752500758D0075DA
:1021B3008B00754100900025E0C394035008900004
:1021C30025E004F080067403900025F0900025E0DC
:1021D300B40306E5B554FEF5B5AE27AF28EFD394A7
:1021E30010EE9427401CC2CA75CD0075CC0075282B
:1021F30000752700D2CA754300752A00752900753A
:052203004700020B463C
:103F82000000010001320164019601960200021252
:103F920002240200020003000340038003C0040065
:103FA2000440048004C00500060006000600060066
:103FB200060006000600060000FF013101630195BC
:103FC20001FF01FF0211022302FF02FF02FF033F72
:103FD200037F03BF03FF043F047F04BF04FF05FF09
:103FE20006FF06FF06FF06FF06FF06FF06FF06FFA7
:10223200900043E090083DF090004AE090083EF0A4
:1022420090004BE090083FF090004EE0900840F084
:1022520090004FE0900841F0900052E0900842F068
:10226200900053E0900843F090005EE0900844F044
:10227200900060E0900845F0900064E0900846F01D
:10228200900066E0900847F0900067E0900848F000
:10229200900068E0900849F0900069E090084AF0E8
:1022A20090006CE090084BF090006DE090084CF0CC
:1022B20090006FE090084DF0900070E090084EF0B2
:1022C20090007CE090084FF090007DE0900850F084
:1022D20090007EE0900851F090007FE0900852F06C
:1022E200900080E0900853F0900081E0900854F054
:1022F200900082E0900855F0900083E0900856F03C
:10230200900085E0900857F0900086E0900858F021
:10231200900087E0900859F0900088E090085AF009
:10232200900126E090085BF0900127E090085CF0B5
:10233200900128E090085DF02290083AE4F0A3F0C2
:10234200755D00755C00756700756800C20DD20E80
:1023520075610075600075633C756200756E00758D
:102362006F00756C0022750B00750A00AE0AAF0B88
:10237200AC08AD09EDC39FEC9E401674FF124043BA
:1023820075CF01780B740126F6500418E436F65026
:10239200DB22C2AF75D900758F0375B7A575B7F18A
:1023A20090F800E4F0758F0175B7A575B7F1E557A0
:1023B20090F800F075B7A575B7F190F801E4F075E3
:1023C200B7A575B7F1900879E090F802F075B7A556
:1023D20075B7F190087DE090F803F075B7A575B771
:1023E200F190087AE090F804F075B7A575B7F1900E
:1023F200087BE090F805F075B7A575B7F190087CF9
:10240200E090F806F075B7A575B7F190087EE090F8
:10241200F807F0758F0075D940D2AF2290083CE0E2
:10242200B4AB61C2AF75D90075B62275F522758F4E
:102432000375B7A575B7F1740090F600F0758F01BA
:10244200755900755800AE58AF59743BBE00279FAE
:10245200402475B7A575B7F190083D12001EE0FC47
:1024620090F60012001EECF07859740126F6500422
:1024720018E436F650D0758F0075F51175B62075D3
:10248200D940D2AF22C2AF75D90075F52275590075
:10249200755800AE58AF59743BBE00229F401F9042
:1024A200F60012001EE493FC90083D12001EECF0B0
:1024B2007859740126F6500418E436F650D575F5AD
:1024C2001175D940D2AF2290083CE0B4AA02800331
:1024D200022606C2AF75D90075B62275F522758F30
:1024E2000375B7A575B7F1740090EE00F075B7A546
:1024F20075B7F1740090F000F075B7A575B7F17477
:102502000090F200F075B7A575B7F1740090F40071
:10251200F0758F01755900755800AE58AF5974FFA8
:10252200C39F74019E402475B7A575B7F190003A18
:1025320012001EE0FC90EE0012001EECF0785974BE
:102542000126F6500418E436F650CF755900755836
:1025520000AE58AF5974FFC39F74019E402475B7F3
:10256200A575B7F190023A12001EE0FC90F000123D
:10257200001EECF07859740126F6500418E436F681
:1025820050CF755900755800AE58AF5974FFC39FAC
:1025920074019E402475B7A575B7F190043A1200F4
:1025A2001EE0FC90F20012001EECF0785974012635
:1025B200F6500418E436F650CF755900755800AE3F
:1025C20058AF5974FFC39F74019E402475B7A57517
:1025D200B7F190063A12001EE0FC90F40012001EC1
:1025E200ECF07859740126F6500418E436F650CF10
:1025F200758F0075F51175B62075D940D2AF743A52
:1026020090073AF02290083CE0B4AA028003022725
:1026120044C2AF75D90075B62275F522758F037560
:10262200B7A575B7F1740090E600F075B7A575B758
:10263200F1740090E800F075B7A575B7F1740090D9
:10264200EA00F075B7A575B7F1740090EC00F0756B
:102652008F01755900755800AE58AF5974FFC39F6A
:1026620074019E402475B7A575B7F190003A120027
:102672001EE0FC90E60012001EECF0785974012670
:10268200F6500418E436F650CF755900755800AE6E
:1026920058AF5974FFC39F74019E402475B7A57546
:1026A200B7F190023A12001EE0FC90E80012001E00
:1026B200ECF07859740126F6500418E436F650CF3F
:1026C200755900755800AE58AF5974FFC39F740115
:1026D2009E402475B7A575B7F190043A12001EE02A
:1026E200FC90EA0012001EECF07859740126F650B4
:1026F2000418E436F650CF755900755800AE58AF3D
:102702005974FFC39F74019E402475B7A575B7F134
:1027120090063A12001EE0FC90EC0012001EECF053
:102722007859740126F6500418E436F650CF758FA6
:102732000075F51175B62075D940D2AF743A90077D
:102742003AF02290083CE0B4AA028003022882C236
:10275200AF75D90075B62275F522758F0375B7A5C9
:1027620075B7F1740090DE00F075B7A575B7F17416
:102772000090E000F075B7A575B7F1740090E20023
:10278200F075B7A575B7F1740090E400F0758F018C
:10279200755900755800AE58AF5974FFC39F740144
:1027A2009E402475B7A575B7F190003A12001EE05D
:1027B200FC90DE0012001EECF07859740126F650EF
:1027C2000418E436F650CF755900755800AE58AF6C
:1027D2005974FFC39F74019E402475B7A575B7F164
:1027E20090023A12001EE0FC90E00012001EECF093
:1027F2007859740126F6500418E436F650CF75590C
:1028020000755800AE58AF5974FFC39F74019E40C3
:102812002475B7A575B7F190043A12001EE0FC903A
:10282200E20012001EECF07859740126F6500418EA
:10283200E436F650CF755900755800AE58AF59744A
:10284200FFC39F74019E402475B7A575B7F190062A
:102852003A12001EE0FC90E40012001EECF07859DF
:10286200740126F6500418E436F650CF758F0075C1
:10287200F51175B62075D940D2AF743A90073AF087
:102882002290083CE0B4AA0280030229C0C2AF75BC
:10289200D90075B62275F522758F0375B7A575B780
:1028A200F1740090D600F075B7A575B7F174009079
:1028B200D800F075B7A575B7F1740090DA00F0751D
:1028C200B7A575B7F1740090DC00F0758F017559EA
:1028D20000755800AE58AF5974FFC39F74019E40F3
:1028E2002475B7A575B7F190003A12001EE0FC906E
:1028F200D60012001EECF07859740126F650041826
:10290200E436F650CF755900755800AE58AF597479
:10291200FFC39F74019E402475B7A575B7F190025D
:102922003A12001EE0FC90D80012001EECF078591A
:10293200740126F6500418E436F650CF7559007526
:102942005800AE58AF5974FFC39F74019E4024755E
:10295200B7A575B7F190043A12001EE0FC90DA00B8
:1029620012001EECF07859740126F6500418E43671
:10297200F650CF755900755800AE58AF5974FFC361
:102982009F74019E402475B7A575B7F190063A125F
:10299200001EE0FC90DC0012001EECF0785974017D
:1029A20026F6500418E436F650CF758F0075F511EF
:1029B20075B62075D940D2AF743A90073AF022C268
:1029C200AF75D90075F522755900755800AE58AF2C
:1029D2005974FFC39F74019E401F90EE0012001EA7
:1029E200E493FC90003A12001EECF0785974012630
:1029F200F6500418E436F650D4755900755800AEF6
:102A020058AF5974FFC39F74019E401F90F000128B
:102A1200001EE493FC90023A12001EECF078597406
:102A22000126F6500418E436F650D475590075584C
:102A320000AE58AF5974FFC39F74019E401F90F2BD
:102A42000012001EE493FC90043A12001EECF0788F
:102A520059740126F6500418E436F650D47559001C
:102A6200755800AE58AF5974FFC39F74019E401F42
:102A720090F40012001EE493FC90063A12001EEC41
:102A8200F07859740126F6500418E436F650D475DD
:102A9200F51175D940D2AF740090006EF0740190B8
:102AA2000044F0743A90073AF022C2AF75D900752B
:102AB200F522755900755800AE58AF5974FFC39F7F
:102AC20074019E401F90E60012001EE493FC9000E9
:102AD2003A12001EECF07859740126F6500418E4FC
:102AE20036F650D4755900755800AE58AF5974FF78
:102AF200C39F74019E401F90E80012001EE493FCE5
:102B020090023A12001EECF07859740126F6500435
:102B120018E436F650D4755900755800AE58AF59BE
:102B220074FFC39F74019E401F90EA0012001EE4CE
:102B320093FC90043A12001EECF07859740126F6C8
:102B4200500418E436F650D4755900755800AE5842
:102B5200AF5974FFC39F74019E401F90EC00120096
:102B62001EE493FC90063A12001EECF078597401B0
:102B720026F6500418E436F650D475F51175D9408E
:102B8200D2AF740090006EF07402900044F0743A78
:102B920090073AF022C2AF75D90075F52275590037
:102BA200755800AE58AF5974FFC39F74019E401F01
:102BB20090DE0012001EE493FC90003A12001EEC1C
:102BC200F07859740126F6500418E436F650D4759C
:102BD2005900755800AE58AF5974FFC39F74019ED7
:102BE200401F90E00012001EE493FC90023A120093
:102BF2001EECF07859740126F6500418E436F650AB
:102C0200D4755900755800AE58AF5974FFC39F74FC
:102C1200019E401F90E20012001EE493FC90043AD1
:102C220012001EECF07859740126F6500418E436AE
:102C3200F650D4755900755800AE58AF5974FFC399
:102C42009F74019E401F90E40012001EE493FC90CA
:102C5200063A12001EECF07859740126F650041858
:102C6200E436F650D475F51175D940D2AF740090A0
:102C7200006EF07403900044F0743A90073AF02228
:102C8200C2AF75D90075F522755900755800AE5856
:102C9200AF5974FFC39F74019E401F90D60012006B
:102CA2001EE493FC90003A12001EECF07859740175
:102CB20026F6500418E436F650D4755900755800BB
:102CC200AE58AF5974FFC39F74019E401F90D80045
:102CD20012001EE493FC90023A12001EECF07859A6
:102CE200740126F6500418E436F650D4755900756E
:102CF2005800AE58AF5974FFC39F74019E401F9095
:102D0200DA0012001EE493FC90043A12001EECF06A
:102D12007859740126F6500418E436F650D47559E1
:102D220000755800AE58AF5974FFC39F74019E409E
:102D32001F90DC0012001EE493FC90063A12001E63
:102D4200ECF07859740126F6500418E436F650D4A3
:102D520075F51175D940D2AF740090006EF074040D
:102D6200900044F0743A90073AF022E568640460F7
:102D720006E59964FF60028031A20D4004D20D8005
:102D820027E568600874E62568900024F0E567602E
:102D92000874F02567900024F0E568B4010280FE13
:102DA200756800756700C20D8002C20DE568903A31
:102DB200A7F8282873756800E599B4FF03756701C1
:102DC200E599B4FE03756702E599B4FD03756703DF
:102DD200E599B4FC03756704E599B4FA03756705D0
:102DE200E599B4FB067568011205EEE599B4F9069A
:102DF2007568041205EEE599B4F7411205EEC29C1E
:102E020074AB90083CF012241E74AA90083CF0E5C2
:012E12004976
:033AA700022DB736
:102E1300903B07F828287380121224C9800D1226CC
:0B2E2300078008122745800312288357
:0F3B0700022E1A022E1C022E21022E26022E2B17
:102E2E0090083CE4F0D29C7568007567007599F7C0
:102E3E00E599D394E54007E599C394F040028016D6
:102E4E008599697568027E017F00E569C394E61273
:102E5E0040718E5E8F5F90083AE4F0A3F0E599D34F
:102E6E0094C44007E599C394E64002802885996989
:102E7E0075680374E5C39569F55F755E00AE5EAF68
:102E8E005F903F8212002EE493F874019390083AFB
:102E9E00C8F0A3C8F0D29902318290083AE0FEA39E
:102EAE00E0FF90003A12001EE599F090083A1200E9
:102EBE000E90083AE0FEA3E0FFEFB40106EEB40771
:102ECE00028003022F9090073AE0B43C0280030286
:102EDE002F901207FCA206B35005A207B340028042
:102EEE0053C29C120088120282900126E090085B69
:102EFE00F0900127E090085CF0900128E090085DCA
:102F0E00F074AB90083CF012241E74AA90083CF0AA
:022F1E00E54983
:033AAA00022EA841
:102F2000903B16F828287380121224C9800D1226AF
:0B2F3000078008122745800312288349
:0F3B1600022F27022F29022F2E022F33022F38C2
:102F3B0090083CE4F08043C29C122232740090084B
:102F4B005BF0740090085CF0740090085DF074AB5B
:102F5B0090083CF012241E74AA90083CF01224C96D
:102F6B00122607122745122883D29C7599FB74648D
:102F7B00F50975080012236880FED29C75680075F0
:102F8B0067007599FB02318290083AE0FEA3E0FFDF
:102F9B00EF4E700685995D755C0090083AE0FEA3D4
:102FAB00E0FF74016F4E701BAC5CAD5DAA5EAB5F56
:102FBB00ED2BFBEC3AFA8A068B0790003A12001EB7
:102FCB00E599F090083A12000E90083AE0FEA3E063
:102FDB00FF74026F4E700C1202828569997568003E
:102FEB0075670002318290083AE0FEA3E0FF900083
:102FFB003A12001EE599F090083A12000E90083A2A
:10300B00E0FEA3E0FFAC5EAD5F8F028E038C068DFE
:10301B0007903FBA12002EE493F9740193FEEAD3A2
:10302B009EEB9940098569997568007567000231B7
:10303B008290083AE0FEA3E0FF90003A12001EE5F2
:10304B0099F090083A12000E90083AE0FEA3E0FFC8
:10305B00EFB40006EEB40102800302318290001837
:10306B00E0D394C7400B900018E0C394C8F56A8076
:10307B001A900018E0D39463400B900018E0C394AF
:10308B0064F56A8006900018E0F56AE56A75F0024F
:10309B00A4FFAEF08F66EF90003A124089EFFCE090
:1030AB00FDEC90003D124089EDFCE0FDEC2DB56A86
:1030BB000280030231730FEF90003A124089E566EC
:1030CB00FFE0FCEF90003E124089ECFFE0FCEFC309
:1030DB009CB56A028003023173E56690003C124096
:1030EB0089E566FFE0FCEF90003F124089ECFFE0C2
:1030FB00FCEF2CB56A72E566900040124089E0C384
:10310B00956A900879F0E566900041124089E0C31A
:10311B00956A90087AF0E566900044124089E0C306
:10312B00956A90087BF0E566900045124089E0C3F4
:10313B00956A90087CF0E566900046124089E0C3E2
:10314B00956A90087DF0E566900047124089E0C3D0
:10315B00956A90087EF01223947599F97464F509B9
:10316B0075080012236880FE7599FF7464F5097564
:07317B00080012236880FE2A
:093AAD00022F93022FF102303CBC
:1031820022E567903AB6F82828730232C390083ACB
:10319200E0FEA3E0FF90000812001EE0F5999008FF
:1031A2003A12000E90083AE0FEA3E0FF741C6F4E44
:1031B20070037567000232C38550990232C39008CA
:1031C2003AE0FEA3E0FF90003A12001EE0F599EF0C
:1031D200B40107EEB4070375670090083A12000EB7
:0731E2000232C390083BE03C
:0F3AB60002318C02318F0231BA0231C00231E588
:1031E900903B25F82828738524990232B8852A99B5
:1031F9000232B8853B990232B8853D990232B885C9
:1032090044990232B8854F990232B88548990232F9
:10321900B88549990232B8756B00900055E070067F
:10322900900054E060028016A2A44006E56B4404B5
:10323900F56BA2A54006E56B4402F56B801A900078
:1032490035E0B40106E56B4410F56B900034E0B449
:103259000106E56B4420F56BA203B34006E56B4418
:1032690001F56BA205B34006E56B4408F56B856B68
:1032790099803CA20EB340077599FAC20E8017A235
:103289000AB3400575990F800B900024E0F59990D9
:103299000024E4F0C20A8017853A99801285409982
:0F32A900800D856C9980087599FC80037567000E
:103B25000231F00231F60231FC02320202320802A1
:103B3500320E02321402321A02322002327C023272
:0D3B4500A10232A60232AB0232B00232B54C
:0B32B80090083A12000E800312023B47
:033AC5000232C00A
:1032C30022E50875F003A4FFAEF0EF241AF509E533
:1032D3000904F50AE5092402F50BE50990003A1201
:1032E3004089E0903AC8F8282873802185246480B7
:1032F3001C852A648017853B648012853D64800D9C
:0D3303008544648008854864800385496422
:103AC8000232ED0232EF0232F40232F90232FE0221
:083AD800330302330802330D31
:10331000E50A90003A124089E50BFEE0FFEE9000CE
:103320003A124089EFFEE0FFEED39F400302341EC5
:10333000E50990003A124089E0D394044051E50A2F
:1033400090003A124089E0D39564500EE50B90004E
:103350003A124089E0C395645002800AE508F50CF2
:10336000D39210120048E50A90003A124089E0D347
:103370009564500EE50B90003A124089E0C39564C5
:10338000500AE508F50CC3921012004802341BE500
:103390000990003A124089E0B40432E50B90003AFB
:1033A000124089E0C39564500AE508F50CD39210E9
:1033B000120048E50A90003A124089E0D395644033
:1033C0000AE508F50CC39210120048804EE50A90F9
:1033D000003A124089E0C39564500EE50B90003A24
:1033E000124089E0D395645002800AE508F50CD3B9
:1033F0009210120048E50A90003A124089E0D395F5
:1034000064500EE50B90003A124089E0C395645079
:103410000AE508F50CC39210120048023509E509C7
:1034200090003A124089E0D394044051E50A90009C
:103430003A124089E0C39564400EE50B90003A12C1
:103440004089E0D395644002800AE508F50CC392F8
:1034500010120048E50A90003A124089E0C39564D2
:10346000400EE50B90003A124089E0D39564400A83
:10347000E508F50CD39210120048023509E50990D1
:10348000003A124089E0B40432E50A90003A124052
:1034900089E0C39564500AE508F50CC39210120048
:1034A00048E50B90003A124089E0D39564400AE564
:1034B00008F50CD39210120048804EE50A90003AAD
:1034C000124089E0C39564400EE50B90003A12402B
:1034D00089E0D39564400AE508F50CD392101200F8
:1034E00048E50A90003A124089E0D39564400EE521
:1034F0000B90003A124089E0C395644002800AE5CF
:1035000008F50CC3921012004822E56D903AE0F8DD
:10351000282873023A947E017F00E5BE124071E5CF
:10352000BD2FFF50010E8E5A8F5B900066E0B401F4
:103530000F7E0F7FFFAC5AAD5B1200038E5A8F5B7C
:10354000900065E0B40245AE5AAF5B900000E0FC2D
:10355000A3E0FDEDD39FEC9E400A900000E55AF0F9
:10356000A3E55BF0AE5AAF5B900002E0FCA3E0FD88
:10357000EFD39DEE9C400A900002E55AF0A3E55B74
:10358000F0AE5AAF5B74041240638F3B900065E06D
:103590007058AE5AAF5B900000E0FCA3E0FDEFD3A3
:1035A0009DEE9C40091200038E5A8F5B8006755B6E
:1035B00000755A00900064E0700674FF900064F09B
:1035C000AE5AAF5B7410124071900064E08E048FAD
:1035D00005FF1240538C5A8D5B7400D39D74019C7F
:1035E0004005855B3B8003753BFFE53B75F00AA416
:1035F000FFAEF074198E048F05FF1240538D3CED21
:103600002561FFAE6050010E74011240638F3C854E
:103610003C61756000EFD394624003753C6290009A
:103620005EE07006900052E060028006756D050253
:10363000350A75BB17023A94023A947E017F00E581
:10364000BE124071E5BD2FFF50010E8E5A8F5B9068
:10365000005EE0B4017AE56345626025AC62AD636B
:103660001DBDFF011C8F028E038C068D07903B52FF
:1036700012002EE493FE740193FFEFC39AEE9B4079
:10368000028005786212409BAE62AF6374B3BE00E5
:1036900021D39F401DAC5AAD5B0FBF00010E903B84
:1036A0005212002EE493FE740193FFEDC39FEC9E33
:1036B00040028005786212003FAE62AF6390006006
:1036C000E012407174648E048F05FF1240538D3DEB
:1036D000E570B40129AE5AAF5BEFD39400EE9408C5
:1036E000400F900052E0B40104C2058002D2058070
:1036F0000D900052E0B40104D2058002C20575BBF2
:1037000016023A94023A947E017F00E5BE1240719F
:10371000E5BD2FFF50010E8E5A8F5B90005EE0B426
:10372000027AE56345626025AC62AD631DBDFF01B1
:103730001C8F028E038C068D07903CBC12002EE479
:1037400093FE740193FFEFC39AEE9B4002800578CD
:103750006212409BAE62AF6374B3BE0021D39F4040
:103760001DAC5AAD5B0FBF00010E903CBC12002E89
:10377000E493FE740193FFEDC39FEC9E400280052D
:10378000786212003FAE62AF63900060E012407159
:1037900074648E048F05FF1240538D3DE570B402B2
:1037A00029AE5AAF5BEFD39400EE9408400F90001F
:1037B00052E0B40104C2058002D205800D9000528F
:1037C000E0B40104D2058002C20590005EE07003FF
:1037D000753D00900052E07002C20575BB1F023AB1
:1037E00094023A947E017F00E5BE124071E5BD2F40
:1037F000FF50010E8E5A8F5B740912407174E68E71
:10380000048F05FF1240538C398D3AE56E2DFD5023
:10381000010C74018C068D071240638E398F3A8536
:103820003A6E75BB19023A94023A947E017F00E524
:10383000BE124071E5BD2FFF50010E8E5A8F5B7492
:10384000041240638F4090006CE0B40102800302D8
:103850003901756600756600E566D394074003027A
:1038600038F7E56690002C124089E0D39540501A55
:10387000E56690002C124089E0F4042540FEE566E0
:1038800090087F124089EEF08017E56690002C12B8
:103890004089E0C39540FEE56690087F124089EEBE
:1038A000F0E566C394044009900070E0C39566504B
:1038B0003BE5666029E56690087F124089FEE0FFDF
:1038C000EE900887E0D39F4013E56690087F124092
:1038D00089E0900887F0E566900888F0800E9008EF
:1038E0007FE0900887F07400900888F07866740193
:1038F00026F64003023858900888E0F4042408F5BE
:103900004890006CE0D394014033E540D3946E407E
:1039100004D20F8002C20F75480590006CE0B4021B
:1039200005A20FB34002800375480790006CE0B415
:103930000306A20FB3B340028003754807E56F6525
:10394000486008E54404F54585486FE548B4070834
:10395000E5B54480F5B58006E5B5547FF5B5E54895
:1039600064066005E548B40808E5B54410F5B5807F
:1039700006E5B554EFF5B575BB13023A94023A94D7
:103980007E017F00E5BE124071E5BD2FFF50010EA4
:103990008E5A8F5B74041240638F6C90006DE0B49C
:1039A00002028003023A8F756600756600E566D3F1
:1039B00094034003023A3CE566900028124089E0F7
:1039C000D3956C501AE566900028124089E0F40403
:1039D000256CFEE566900889124089EEF08017E5B7
:1039E00066900028124089E0C3956CFEE566900859
:1039F00089124089EEF0E5666029E5669008891233
:103A00004089FEE0FFEE90088DE0D39F4013E5660D
:103A1000900889124089E090088DF0E56690088E44
:103A2000F0800E900889E090088DF0740090088E68
:103A3000F07866740126F640030239AD90006EE01E
:103A4000704DE52A45296036E549C39403500A9034
:103A5000088EE004C394034002800790088EE004BF
:103A6000F549E549D39402400A90088EE004D394C6
:103A7000025002800790088EE004F54980119008FA
:103A80008EE004F549E549D3940440037549017576
:043A9000BB188000DF
:103AE00002351302351602363802363B023704021D
:103AF00037070237E10237E402382802382B02394F
:073B00007D023980023A94B6
:103A9400E56D75F00284AFF07E00EF4E7002D2EC5B
:033AA400056D228B
:094089002582F582500205832214
:10002E00EF2F500205832582F582E5833E2EF58360
:01003E00229F
:08000300C3EF9DFFEE9CFE22FD
:08003F000806B60002180622B3
:0D000E00A3E004F0700612407FE004F02231
:08409B000816B6FF02181622F8
:0E406300048007C3CE13CECF13CFD5E0F622D4
:103EA100BC000FBE0008ED8FF084FFADF022E4FEF0
:103EB100FF22BE000DEF60FE54F0606F20E70302A9
:103EC1003F57EAC0E0EBC0E078017A0075F001EEFF
:103ED10020E710EF25E0FFEE33FE0AC5F023C5F021
:103EE10030E7F0EA5407F9096A7A007B00600108BB
:103EF100C3EC9E40167004ED9F4010ED9FFDEC9EBB
:103F0100FCE5F0CA4ACA03F5F08005E5F003F5F0D7
:103F1100C3EE13FEEF13FFD9D77908CACBCAD8D0A5
:103F2100EAFEEBFFD0E0FBD0E0FA22EC8FF084FC5C
:103F3100ED54F045F0C48FF084FEEDC454F045F02B
:103F4100C48FF084FDEEC4FE54F02DFFEE540F3CFF
:103F5100FEADF07C0022790078008FF0EC7E082025
:103F6100E70DC3CD33CD33C933C9C833C8DEF084BF
:103F710049F9E5F08FF0BE00E6FD7C00E9FFE8FEBF
:013F8100221D
:0E407100F88FF0A4FFE5F0CE88F0A42EFE221A
:10404300600D782B02404D007830D8FED5E0F82281
:10405300EEC0E07E00123EA1EFFDEEFCD0E0FE22BA
:03000B00023FF2BF
:03001B0002400D93
:03002B0002402868
:0300000002409229
:0940920075817175D00002080E61
:0B001E00E5822FF582E5833EF583228A
:0A407F000582D58202158315822206
:103FF200C0E0C0F0C083C082C0D075D000120803F8
:10400200D0D0D082D083D0F0D0E032C0E0C0F0C0B7
:1040120083C082C0D075D000120806D0D0D082D022
:1040220083D0F0D0E032C0E0C0F0C083C082C0D004
:1040320075D000120809D0D0D082D083D0F0D0E061
:01404200324B
:00000001FF
